:020000000528D1
:1000080009008316043085008B3081007F30900012
:1000180054309F00831207309900013018202B209C
:10002800FB3E031818201328013EA100003CA20043
:1000380005162520A10B1D2805122520A20B212815
:1000480008000C30A3006400A30B27280800023026
:100058002D280339A5000310A50DA50D2508033883
:100068009F00000064009F1836281E080800A200A0
:0C007800A100A10B3D28A20B3C280800B1
:02400E00AC0103
:00000001FF
